:100000000C94F4020C9438030C9438030C943803C9
:100010000C9438030C9438030C9438030C94380374
:100020000C9438030C9438030C94320E0C94040F87
:100030000C9438030C9438030C9438030C94380354
:100040000C9438030C940E230C9438030C9438034E
:100050000C9438030C94A11C0C9438030C943803B2
:100060000C9438030C9438030C9438030C94380324
:100070000C9438030C9438030C9438030C94380314
:100080000C9438030C9438030C9438030C94380304
:100090000C9438030C9438030C9438030C943803F4
:1000A0000C9438030C9438030C9438039E05A40573
:1000B000AA05B005B605BB05C005CA05CF05C5052F
:1000C000D405D905DE05E305E805ED05710F930FAD
:1000D0008110930F8110D80FFB0F81105010631007
:1000E00032133213611361139713B713E814E81432
:1000F000C213E81472147214D914E814E814E21448
:100100007F147F147F147F147F147F147F147F1457
:100110007F147F147F147F147F147F147F147F1447
:1001200091149E14A514AC14B61401E10126022604
:100130000127022702E101330233000111021101FC
:10014000080208011A021A012C022C000138023898
:100150000138023801E101170217011202120107EA
:1001600002070112021202E1012C022C0001050219
:1001700005011502150108020801040204010E021E
:100180000E01330233000111021101180218010F90
:10019000020F010F020F00011502150108020801EC
:1001A000170217011802180115021501110211009A
:1001B00001090209010F020F0112021201040204D7
:1001C00001170217012C022C00010C020C01110274
:1001D0001101170217012C022C0001050205011262
:1001E000021201120212010F020F012C022C000157
:1001F0001602160117021701150215010C020C0157
:10020000110211010A020A012C022C000119021923
:100210000104020401150215012C022C000119022F
:100220001901120212010C020C01070207012C0233
:100230002C00010602060112021201110211011620
:10024000021601170217012C022C000116021601DA
:100250001702170104020401170217010C020C0116
:10026000060206012C022C000113021301150215CF
:10027000010C020C011902190104020401170217F2
:1002800001080208012C022C0001130213011802BC
:100290001801050205010F020F010C020C010602F4
:1002A00006012C022C000000F0A1260227022F02DA
:1002B00030022B7100001E00140004001D74360271
:1002C00019011F001A0016001B0037022C722000B3
:1002D00008000700060031022878210015000900F7
:1002E000190024020601220017000A000500000080
:1002F000374134022A0000003800000036001601A1
:100300004C000000330000004A0023001C000B00DA
:10031000110000004D41240018000D0010002E00B7
:10032000520025000C000E0034002E022878260012
:1003300012000F001E022D002C72270013002D0248
:100340003802250251002F0030001C011D0101540C
:10035000000029002B0001000100010000003A000C
:100360000A300B300100E30001003B000C300D307F
:100370000100E20001003C0010300F300E3001009F
:1003800001003D00113012301330010001003E0029
:100390001430153016300000010035000100000057
:1003A000310000001B01B200010000003502000016
:1003B00001003F00173018301930000001004000E4
:1003C0000100010001004B0001004100010001009B
:1003D00001004E004F0042000100010001004900F1
:1003E00050004300010001000100460001004400EC
:1003F00045000100010001000000160345007200E5
:1004000067006F0044006F007800200045005A002C
:10041000000016034500720067006F0044006F0083
:100420007800200045005A00000004030904090276
:100430006D00040100A0FA0904000001030101009D
:10044000092111010001223F000705810308000A6C
:100450000904010001030102000921110100012228
:100460004D000705820308000A0904020001030089
:10047000000009211101000122360007058303084D
:10048000000A090403000103000000092111010012
:100490000122390007058403100001120110010038
:1004A000000008EDFE07130100010200010501092B
:1004B00006A101050719E029E71500250195087532
:1004C000018102050819012905950575019102951B
:1004D000017503910105071900297715002501957C
:1004E0007875018102C005010980A101850216010C
:1004F0000026B7001A01002AB70075109501810087
:10050000C0050C0901A1018503160100269C021AF1
:1005100001002A9C02751095018100C005010902A5
:10052000A1010901A10005091901290515002501ED
:100530009505750181029501750381010501093059
:1005400009311581257F95027508810609381581C5
:10055000257F950175088106050C0A38021581254D
:100560007F950175088106C0C005010906A1010536
:100570000719E029E7150025019508750181029505
:100580000175088101050819012905950575019175
:10059000029501750391010507190029FF15002532
:1005A000FF950675088100C00000000000000000F3
:1005B000000000010204060A0F17202C3A4A5D7160
:1005C000879DB3C7DAE9F5FCFFFCF5E9DAC7B39D0F
:1005D00087715D4A3A2C20170F0A060402010000B9
:1005E000000000000000000011241FBECFEFDAE081
:1005F000DEBFCDBF04B603FE24C08091FB01909105
:10060000FC01A091FD01B091FE018730904BA74005
:10061000B04BB9F41092FB011092FC011092FD0155
:100620001092FE0114BE84B7877F84BF88E10FB6A5
:10063000F89480936000109260000FBEE0E0FFE34A
:10064000099511E0A0E0B1E0EAEAF9E402C0059002
:100650000D92A433B107D9F711E0A4E3B1E001C0D2
:100660001D92AB3FB107E1F70E94760B0C94D324A7
:100670000C9400001092B9008AE08093B8000895AD
:1006800094EA9093BC009091BC0097FFFCCF9091AE
:10069000B900987F983021F0903111F081E00895F1
:1006A0008093BB0084E88093BC008091BC0087FFEE
:1006B000FCCF8091B900887F883111F0803471F7C8
:1006C00080E0089584E98093BC008091BC0084FDA3
:1006D000FCCF08958093BB0084E88093BC00809198
:1006E000BC0087FFFCCF9091B900987F81E09832E1
:1006F00009F480E0089584E88093BC008091BC00F8
:1007000087FFFCCF8091BB0008958091010181118A
:1007100015C080E40E9440038093010181110CC048
:1007200082E10E946A0380930101811105C08FEF6D
:100730000E946A03809301010E94620384B1807F5A
:1007400084B985B1807F85B98AB1837F8AB98BB13D
:10075000837F8BB93E98469808950E944005809308
:1007600001010E94850380B38C7080BB81B3836FCD
:1007700081BBA5E3B1E0E3E4F1E08EE08E0F1192DE
:100780001D928E13FCCF0C942A05BF92CF92DF925C
:10079000EF92FF920F931F93CF93DF93809101010C
:1007A000882379F0809134018F5F80933401811127
:1007B00008C00E94400580930101811102C00E947F
:1007C000D20405E311E0C0E0D0E0DD24D39482E060
:1007D000C82EEE24E394F12CC730D10500F58091AA
:1007E0000101811164C080E40E94400380930101F3
:1007F000811112C082E10E946A038093010181117C
:100800000BC0C7010C2E01C0880F0A94EAF780952F
:100810000E946A03809301010E94620348C0CA30AB
:10082000A1F028F4C83059F0C93061F005C0CC30CF
:1008300089F070F0CD3089F0209A289810C0219A64
:1008400029980DC0229A2A980AC0239A2B9807C08B
:10085000529A01C0539A5B9802C03E9A469890EA19
:100860009A95F1F79FB1799902C082E001C080E0CA
:1008700091709D25982B7C9902C084E001C080E096
:10088000892B7D9902C038E001C030E0832B7E992E
:1008900002C020E101C020E0822B9FB19095991FFA
:1008A0009927991F9295990F907E892B0FC080915F
:1008B0000101811149C080E40E944003809301013D
:1008C000882379F1B12C0E9462038B2DF80190816D
:1008D000981719F08083C09200010E948503219629
:1008E0000F5F1F4FCE30D10509F076CF8091000108
:1008F000882361F1815080930001882339F08FE9CA
:100900009FE00197F1F700C0000020C0A3E4B1E030
:10091000E5E3F1E0CF01825F91919D938E13FCCFCF
:1009200015C083E10E946A03809301018111CACF3F
:1009300081E40E944003809301018111C3CF0E9492
:100940007B03B82EB094BFCF80E0C0CF0E94D0040C
:1009500081E0DF91CF911F910F91FF90EF90DF9099
:10096000CF90BF900895E82FF0E0ED5BFE4F8081BF
:10097000089508950F931F93CF93DF93C3E4D1E0BD
:1009800010E00C2F025F899190E00E94C71B180FA6
:100990000C13F9CF812FDF91CF911F910F91089503
:1009A0000C94F60556985E9825982D9826982E98C2
:1009B00027982F988FEF90E090938900809388007C
:1009C00090938B0080938A0090938D0080938C008D
:1009D000259A2D9A2FEF80E792E021508040904099
:1009E000E1F700C00000269A2E9A2FEF80E792E0F0
:1009F000215080409040E1F700C00000279A2F9AD4
:100A00002FEF80E792E0215080409040E1F700C056
:100A1000000025982D982FEF80E792E0215080402C
:100A20009040E1F700C0000026982E982FEF80E755
:100A300092E0215080409040E1F700C000002798EC
:100A40002F9856985E9825982D9826982E98279836
:100A50002F98089589EA8093800089E0809381002F
:100A600024982C983F988AB18F748AB96E98479AC7
:100A70008BB1806B8BB9769A0E94D2040C94F505E9
:100A800080E2809301018091510181110EC00E948A
:100A90003A0381E0809351012FEF83ED90E32150E1
:100AA00080409040E1F700C0000080E40E944003D5
:100AB0008093010181112EC00E946A03809301017D
:100AC000811128C00E946A0380930101811122C014
:100AD0008FE30E946A038093010181111BC00E9471
:100AE000620380E40E94400380930101811112C0DF
:100AF0008CE00E946A038093010181110BC00E9467
:100B00006A0380930101811105C08FE30E946A038B
:100B1000809301010E946203809101010895462F94
:100B200050E0FA013A97E031F10508F05BC0EA5A6B
:100B3000FF4FDC0112968C910C948324882309F4D6
:100B400051C089E892E00895882309F44BC088E6F3
:100B500092E00895882309F445C08BE492E008955B
:100B6000882309F43FC082E392E008958823D1F1FD
:100B70008DE192E008958823A9F18CE092E0089538
:100B8000882381F18FEE91E00895882359F18AED51
:100B900091E00895882331F189EC91E0089588234C
:100BA00009F180EB91E008958823E1F087E991E075
:100BB00008958823B9F086E891E00895882391F09C
:100BC0008DE691E00895882369F08CE491E0089522
:100BD000882341F08BE391E00895882319F08AE29D
:100BE00091E0089580E090E0089508956091BD013E
:100BF0007091BE018091BF019091C0010E94D31BF2
:100C000056985E9825982D9826982E9827982F9874
:100C1000813019F0823021F00895259A2D9A089597
:100C2000269A2E9A089581E0089581E008950C9403
:100C3000150608950F931F93CF93DF938C01FC014A
:100C4000C081D181CE010E944C1ABE010E94C30610
:100C5000EC01B8010E941706882309F48DC0F80141
:100C60008281882309F44AC080915D0181111FC0EF
:100C7000C431F0E5DF0709F051C00E94190681E098
:100C800080935D010E946B1C90935C0180935B01DB
:100C90001092540110925601109255011092580171
:100CA0001092570110925A011092590165C080911B
:100CB0005B0190915C010E94771C883C910570F467
:100CC00080915401E82FF0E0EE0FFF1FEB5AFE4F2A
:100CD000D183C0838F5F809354014EC0C43880E5B8
:100CE000D80721F0C538D04501F13AC0F80182811A
:100CF000882341F01092520182E01EC0C438E0E522
:100D0000DE0759F580915201811106C086E20E94EA
:100D1000D61186E20E949E1282E01CC0C438F0E523
:100D2000DF0741F3C538D045D9F4F8018281882323
:100D300031F01092530180E20E94ED121DC08091AB
:100D40005301811106C087E20E94D61187E20E94FA
:100D50009E1280E20E94F4120FC0C538D04529F3DC
:100D600081E08093520180935301C801DF91CF91BC
:100D70001F910F910C94130680E0DF91CF911F918A
:100D80000F910895089596E0799FF001112494E55C
:100D9000899FE00DF11D1124E60FF11DEE0FFF1FDD
:100DA000E655FD4F859194910895880F991FFC0198
:100DB000EA5DFE4F859194910895880F991FFC017B
:100DC000EA55FD4F8591949108950F931F93CF930A
:100DD000DF93EC01811520E3920750F5C11580E205
:100DE000D80708F0C3C0CB3BD10590F4C83AD10571
:100DF00008F06AC0C53AD10508F05BC0C430D1051F
:100E000008F0D0C1219709F0CAC101E010E00AC280
:100E1000CF3FD10511F008F0C5C1C03FD10508F0A2
:100E2000A2C0CE01805E9109089708F4BBC1B7C18A
:100E3000C13090E5D90709F4A2C020F5C0318FE494
:100E4000D80770F4C11590E4D90708F094C0C11513
:100E500021E3D20708F0A3C1DD278E01106CE2C1A7
:100E6000C115D04509F09BC10E9453158FEF94E343
:100E70002CE0815090402040E1F700C000000E942B
:100E8000C61CD0C1C11597E5D90758F4C03121E57A
:100E9000D20708F01CC1C43180E5D80708F475C03A
:100EA0007EC1CE0190578115904108F078C1DF7066
:100EB00073C1C53AD10509F477C1C63AD10509F025
:100EC00076C102E810E4AEC1C83AD10509F472C196
:100ED000C93AD10509F471C1CA3AD10509F470C102
:100EE000CB3AD10509F46FC1CC3AD10509F46EC1F2
:100EF000CD3AD10509F46DC1C03BD10509F46CC1EF
:100F0000CE3AD10509F46BC1CF3AD10509F46AC1D3
:100F1000C13BD10509F469C1C23BD10509F468C1DF
:100F2000C33BD10509F467C1C43BD10509F466C1CF
:100F3000C53BD10509F465C1C63BD10509F464C1BF
:100F4000C73BD10509F463C1C83BD10509F462C1AF
:100F5000C93BD10509F461C1CA3BD10509F460C19F
:100F600000E014E45FC18E0110655CC1CE019F708A
:100F70000E94DD0658C1DF708E01106A53C1809156
:100F8000DA0181608093DA014DC10E946B1E8111EC
:100F900002C00E94511E0E94881E90E09093FB01A7
:100FA0008093FA01C23080E5D80721F48091FA01DC
:100FB000816086C0C43090E5D90721F48091FA01A0
:100FC00082607EC0C63020E5D20721F48091FA010C
:100FD000846076C0C83080E5D80719F48091FA01A2
:100FE00027C0CA3090E5D90721F48091FA018061C9
:100FF00067C0CC3020E5D20721F48091FA018062ED
:101000005FC0CE3080E5D80721F48091FA0180647A
:1010100057C0C03190E5D90721F48091FA0180686A
:101020004FC0C23120E5D20729F48091FA018460D3
:10103000886046C0C33080E5D80721F48091FA016A
:101040008E7F3EC0C53090E5D90721F48091FA012A
:101050008D7F36C0C73020E5D20721F48091FA0198
:101060008B7F2EC0C93080E5D80719F48091FA0132
:1010700026C0CB3090E5D90721F48091FA018F7E0C
:101080001FC0CD3020E5D20721F48091FA018F7D79
:1010900017C0CF3080E5D80721F48091FA018F7B0B
:1010A0000FC0C13190E5D90721F48091FA018F7703
:1010B00007C0C331D04531F48091FA018B7F877F1F
:1010C0008093FA018091FA010E948C1EABC08D2F93
:1010D00099278F70992781309105D9F49E0123704B
:1010E000332702C0880F991F2A95E2F79C688E016A
:1010F00044E0000F111F4A95E1F700271370802B81
:10110000912B53E0CC0FDD1F5A95E1F7C076DD2718
:101110002FC08230910531F4DC2FCC278E01016F76
:10112000106A80C08330910569F4CE0183709927DD
:1011300001E010E002C0000F111F8A95E2F7C8011C
:101140009C680FC084309105B9F4CE018370992753
:1011500001E010E002C0000F111F8A95E2F7C801FC
:101160009A6823E0CC0FDD1F2A95E1F7C07ED77087
:101170008C010C2B1D2B56C08530910531F4DC2FD2
:10118000CC278E01046F106A4DC0069709F04AC043
:10119000CF71DD27DC2FCC278E01106243C000E029
:1011A00010E040C08E013EC001E810E43BC003E8FF
:1011B00010E438C002EE14E435C009EE14E432C085
:1011C0000AEE14E42FC005EB14E42CC006EB14E483
:1011D00029C007EB14E426C00CEC14E423C00DEC8A
:1011E00014E420C003E815E41DC00AE815E41AC0A1
:1011F00002E915E417C004E915E414C001E216E49D
:1012000011C003E216E40EC004E216E40BC005E2CE
:1012100016E408C006E216E405C007E216E402C0C0
:101220000AE216E4C801DF91CF911F910F91089552
:1012300096E0799FF001112494E5899FE00DF11D5E
:101240001124E60FF11DEE0FFF1FE655FD4F8591AE
:101250009491803E9105E0F4803C910558F58133EE
:10126000910509F46FC048F48932910509F463C00F
:101270008A32910509F46DC072C089339105E9F095
:1012800082389105D1F08533910509F44DC067C0CE
:10129000833E910581F138F4803E9105B9F0823E9C
:1012A0009105D9F05CC0863E910561F1873E9105BC
:1012B000A1F155C00E94D50608952091FA0120FDA4
:1012C00002C021FF4CC080EE90E049C08091FA013D
:1012D00080FFF9CF89E390E042C08091FA0182FF5C
:1012E0000EC08091FA0184FF03C080E090E037C017
:1012F00083EE90E034C08091FA0182FFF2CF82EE5B
:1013000090E02DC08091FA0183FF0BC08091FA011B
:1013100084FDEBCF87EE90E022C08091FA0183FF3D
:10132000F5CF86EE90E01BC08091FA0185FF07C0E3
:1013300089E290E014C08091FA0185FFF9CF85E33E
:1013400090E00DC08091FA0186FF07C08AE290E02C
:1013500006C08091FA0186FFF9CF81E390E00E94F8
:10136000E506089508950C94B20980916E010895E0
:10137000CF93DF9300D01F92CDB7DEB79C01809151
:10138000F101843019F593E099833B832A8390938C
:10139000E9008FEF9091E800815095FD06C095ED32
:1013A0009A95F1F700008111F5CF8091E80085FF53
:1013B0000DC040E050E063E070E0CE0101960E9475
:1013C000220C8091E8008E778093E8000F900F90B8
:1013D0000F90DF91CF910895CF93DF9300D01F92AC
:1013E000CDB7DEB72091F101243021F522E0298329
:1013F0009B838A8383E08093E9008FEF9091E800DC
:10140000815095FD06C095ED9A95F1F70000811188
:10141000F5CF8091E80085FF0DC040E050E063E02B
:1014200070E0CE0101960E94220C8091E8008E7738
:101430008093E8000F900F900F90DF91CF91089567
:101440002091F1012430F1F422E02093E9002FEF04
:101450003091E800215035FD06C035ED3A95F1F7A1
:1014600000002111F5CF2091E80025FF0BC040E0DE
:1014700050E065E070E00E94220C8091E8008E77D9
:101480008093E8000895CF93DF93EC019091F101F0
:10149000943009F046C080910C018823D9F08091E6
:1014A0000D018823B9F09093E9008FEF9091E80047
:1014B000815095FD06C095E19A95F1F700008111E4
:1014C000F5CF8091E80085FF2CC040E050E060E15E
:1014D00070E017C081E08093E9008FEF9091E80001
:1014E000815095FD06C095ED9A95F1F700008111A8
:1014F000F5CF8091E80085FF14C040E050E068E03F
:1015000070E0CE010E94220C8091E8008E778093DB
:10151000E80080E1FE01AEE5B1E001900D928A9510
:10152000E1F7DF91CF9108958091F001811109C019
:101530000E94B70D0E94140E8091E2008460809397
:10154000E20008951092F001089508950C94FB2292
:101550000E945C1C0E9401230E94BA100C94B309E3
:1015600042E061EC81E00E94310D42E061EC82E0FA
:101570000E94310D42E061EC83E00E94310D42E1B6
:1015800061EC84E00C94310D8091F301833009F417
:1015900055C030F4813071F0823009F48EC0089566
:1015A0008A3009F47AC08B3009F460C0893009F0C0
:1015B0009CC020C08091F201813A09F096C08091D0
:1015C000E800877F8093E8008091F6019091F70111
:1015D000892B21F460E18EE591E003C060E080E0BA
:1015E00090E070E00E946D0C8091E8008B77809312
:1015F000E80008958091F201813209F076C080916F
:10160000F6019091F701009719F0039709F06DC06A
:101610008091E800877F8093E8008091E80082FD58
:1016200005C08091F1018111F8CF5FC08091F10078
:1016300080936E018091E8008B7753C08091F20116
:10164000813A09F052C08091F6019091F701892BFF
:1016500009F04BC08091E800877F8093E80080917B
:10166000E80080FFFCCF80910C0136C08091F20130
:101670008132D9F58091F6019091F701892BA9F576
:101680008091E800877F8093E8000E94660D80913A
:10169000F40180930C010C9453158091F201813276
:1016A00021F58091E800877F8093E8000E94660D15
:1016B0008091F50180936F0108958091F201813A44
:1016C000A1F48091E800877F8093E8008091E80092
:1016D00080FFFCCF80916F018093F1008091E80042
:1016E0008E778093E8000C94660D089584B7877F09
:1016F00084BF88E10FB6F894809360001092600078
:101700000FBE90E080E80FB6F8948093610090934C
:1017100061000FBE0E9409110E94B70D0E94140EB5
:101720008091E20084608093E20078940E949A1095
:101730000E940B1182E091E00E94B5100E94E92204
:101740008091F101853069F40E94231C8091EF01A2
:101750008823B1F30E944E1C882391F30E940C0C45
:10176000EFCF0E941111ECCF292F33272330310501
:10177000C9F064F42130310581F02230310509F0DF
:1017800043C08DE690E02EE234E042C021323105C4
:10179000F1F02232310541F137C082E190E02BE9CE
:1017A00034E036C099278130910541F082309105AF
:1017B00041F0892B49F5EAE2F4E005C0E2E1F4E00A
:1017C00002C0EAEFF3E0849190E09F0121C0643011
:1017D000D8F4E62FF0E0EE0FFF1FEE5DFE4F208104
:1017E000318189E090E014C0643070F470E0FB0156
:1017F000EE0FFF1FE65EFE4F20813181FB01EA5EA6
:10180000FE4F808190E004C080E090E020E030E076
:10181000FA0131832083089580E189BD82E189BD89
:1018200009B400FEFDCF8091D8008F7D8093D80051
:101830008091E00082608093E0008091E00081FD73
:10184000FCCF0895CF92DF92EF92FF920F931F93F8
:10185000CF93DF93EC018B016A010E94850D81110A
:1018600033C0C114D10439F0F60180819181081B85
:10187000190BC80FD91FE12CF12C0115110519F115
:101880008091E80085FD16C08091E8008E778093F6
:10189000E800C114D10449F0F60180819181E80E7D
:1018A000F91EF182E08285E00FC00E94850D882339
:1018B00021F30AC089918093F10001501109FFEFD3
:1018C000EF1AFF0ADACF80E0DF91CF911F910F91DD
:1018D000FF90EF90DF90CF9008952091F801309124
:1018E000F9012617370748F06115710539F4209181
:1018F000E8002E772093E80001C0B90140E06115AF
:101900007105A9F12091F101222309F443C025308A
:1019100009F442C02091E80023FD40C02091E80076
:1019200022FD32C02091E80020FFE9CF4091F30072
:101930002091F20030E0342BFC01CF0161157105DC
:1019400059F02830310540F481918093F1006150C5
:1019500071092F5F3F4FF1CF41E02830310509F089
:1019600040E02091E8002E772093E800C8CF411195
:10197000C9CF0AC08091F101882361F0853061F000
:101980008091E80083FD0AC08091E80082FFF2CFD9
:1019900080E0089582E0089583E0089581E008954D
:1019A0002091F8013091F9012617370748F06115A9
:1019B000710539F42091E8002E772093E80001C0EA
:1019C000B901FC0120E06115710591F18091F101EF
:1019D000882309F440C0853009F43FC08091E800B5
:1019E00083FD3DC08091E80082FD2FC08091E8001A
:1019F00080FFE9CF2091F3008091F20090E0922BDC
:101A00006115710559F08830910540F424912093B7
:101A1000F1003196615071090196F2CF21E00897EB
:101A200009F020E08091E8008E778093E800CBCF2A
:101A30002111CCCF0AC08091F101882361F085305B
:101A400061F08091E80083FD0AC08091E80082FF88
:101A5000F2CF80E0089582E0089583E0089581E068
:101A60000895982F973058F59093E900981739F01A
:101A70007091EC002091ED005091F00003C0242FF4
:101A8000762F50E021FF19C03091EB003E7F30935C
:101A9000EB003091ED003D7F3093ED003091EB0095
:101AA00031603093EB007093EC002093ED00509385
:101AB000F0002091EE0027FF07C09F5FD3CF8F700B
:101AC0008093E90081E0089580E008958091F2011B
:101AD00087FF11C08091E80082FD05C08091F1016F
:101AE0008111F8CF11C08091E8008B770BC08091F5
:101AF000F101882349F08091E80080FFF8CF8091C0
:101B0000E8008E778093E80008952091E4003091FA
:101B1000E50095E64091EC00842F817040FF22C0E3
:101B20008091E80080FD1CC08091F101882391F034
:101B3000853091F08091EB0085FD10C04091E4006C
:101B40005091E5004217530729F39A01915011F77C
:101B500084E0089582E0089583E0089581E0089587
:101B600080E008954091E80042FFDECF08950E9492
:101B7000250E0E942D0EE0EEF0E0808181608083D2
:101B8000E8EDF0E080818F77808319BCA7EDB0E0AD
:101B90008C918E7F8C9380818F7E80831092F00158
:101BA00008950F931F93CF93DF930E94250E0E94F9
:101BB0002D0EC8EDD0E088818F778883888180687A
:101BC000888388818F7D888319BC1092F1011092DF
:101BD000ED011092EF011092EE0100EE10E0F8011D
:101BE00080818B7F808388818160888342E060E090
:101BF00080E00E94310DE1EEF0E080818E7F8083F5
:101C0000E2EEF0E080818160808380818860808363
:101C1000F80180818E7F8083888180618883DF9155
:101C2000CF911F910F910895E8EDF0E080818F7EB4
:101C30008083E7EDF0E080818160808384E082BF73
:101C400081E08093F0010C94D10DE8EDF0E080810B
:101C50008E7F80831092E20008951092DA00109235
:101C6000E10008951F920F920FB60F9211242F9347
:101C70003F934F935F936F937F938F939F93AF9314
:101C8000BF93EF93FF938091E10082FF0BC080919F
:101C9000E20082FF07C08091E1008B7F8093E1002A
:101CA0000E9499108091DA0080FF1FC08091D800B7
:101CB00080FF1BC08091DA008E7F8093DA008091D4
:101CC000D90080FF0DC080E189BD82E189BD09B4E2
:101CD00000FEFDCF81E08093F1010E94940A05C0CF
:101CE00019BC1092F1010E94A20A8091E10080FFCC
:101CF00019C08091E20080FF15C08091E2008E7FC4
:101D00008093E2008091E20080618093E200809104
:101D1000D80080628093D80019BC85E08093F101DF
:101D20000E94A60A8091E10084FF30C08091E20009
:101D300084FF2CC080E189BD82E189BD09B400FE29
:101D4000FDCF8091D8008F7D8093D8008091E100F5
:101D50008F7E8093E1008091E2008F7E8093E2008D
:101D60008091E20081608093E2008091ED01882300
:101D700011F084E007C08091E30087FD02C081E09C
:101D800001C083E08093F1010E94A80A8091E100E4
:101D900083FF29C08091E20083FF25C08091E1008C
:101DA000877F8093E10082E08093F1011092ED0142
:101DB0008091E1008E7F8093E1008091E2008E7F30
:101DC0008093E2008091E20080618093E20042E033
:101DD00060E080E00E94310D8091F0008860809387
:101DE000F0000E94A50AFF91EF91BF91AF919F91E2
:101DF0008F917F916F915F914F913F912F910F90B4
:101E00000FBE0F901F9018951F920F920FB60F9252
:101E100011242F933F934F935F936F937F938F93EF
:101E20009F93AF93BF93CF93DF93EF93FF93C091B3
:101E3000E900CF708091EC00D82FD17080FDD0E800
:101E40001092E9008091F000877F8093F0007894F1
:101E50000E94480F1092E9008091F0008860809302
:101E6000F000CD2BCF70C093E900FF91EF91DF918F
:101E7000CF91BF91AF919F918F917F916F915F9122
:101E80004F913F912F910F900FBE0F901F9018957B
:101E90001F93CF93DF93CDB7DEB7AA970FB6F89411
:101EA000DEBF0FBECDBFE2EFF1E088E08E0F909174
:101EB000F10091938E13FBCF0E94C40A8091E80039
:101EC00083FF1FC18091F2019091F301492F50E0EF
:101ED0004A30510508F015C1FA01EA59FF4F0C9438
:101EE0008324803881F0823809F00BC18091F6019B
:101EF0008F708093E9008091EB0085FB882780F943
:101F00001092E90006C08091EE019091EF019111CD
:101F100082609091E800977F9093E8008093F100B1
:101F20001092F100C8C0282F2D7F09F0EAC0882345
:101F300019F0823061F0E5C08091F401813009F040
:101F4000E0C0933009F080E08093EF012BC08091D6
:101F5000F401811127C08091F6018F7009F4D1C07E
:101F60008093E9002091EB0020FF1CC0933021F406
:101F70008091EB00806214C09091EB00906190938F
:101F8000EB0021E030E0A90102C0440F551F8A9503
:101F9000E2F74093EA001092EA008091EB0088603B
:101FA0008093EB001092E9008091E800877F86C063
:101FB0008111A7C01091F4011F778091E300807810
:101FC000812B8093E3008091E800877F8093E80075
:101FD0000E94660D8091E80080FFFCCF8091E300B5
:101FE00080688093E300111102C082E001C083E0A9
:101FF0008093F10186C08058823008F082C08091C1
:10200000F4019091F5018C3D53E0950779F583E05B
:102010008A838AE289834FB7F894DE01139620E021
:102020003EE051E2E32FF0E050935700E49120FFAF
:1020300003C0E295EF703F5FEF708E2F90E0EA30C3
:1020400010F0C79601C0C0968D939D932F5F2431E9
:1020500049F74FBF8091E800877F8093E8006AE2EC
:1020600070E0CE0101960E946D0C14C0AE014F5F6E
:102070005F4F6091F6010E94B40BBC01009709F418
:1020800040C09091E800977F9093E80089819A8101
:102090000E94D00C8091E8008B778093E80031C0DB
:1020A000803879F58091E800877F8093E8008091FF
:1020B000ED018093F1008091E8008E778093E80035
:1020C0000E94660D1EC081111CC09091F4019230D7
:1020D000C0F48091E800877F8093E8009093ED0141
:1020E0000E94660D8091ED01811106C08091E30090
:1020F00087FD02C081E001C084E08093F1010E946D
:10210000B00A8091E80083FF0AC08091E800877FD1
:102110008093E8008091EB0080628093EB00AA96A8
:102120000FB6F894DEBF0FBECDBFDF91CF911F91E8
:1021300008950895CF938091F1018823A1F0C09173
:10214000E900CF709091EC00892F817090FD80E8BC
:10215000C82B1092E9008091E80083FD0E94480F8F
:10216000CF70C093E900CF9108959093750180934B
:1021700074010895E0917401F0917501309721F098
:102180000190F081E02D099480E00895E0917401C0
:10219000F0917501309721F00280F381E02D0994D0
:1021A0000895E0917401F0917501309721F0048059
:1021B000F581E02D09940895209172013091730109
:1021C0008217930771F09093730180937201E091ED
:1021D0007401F0917501309721F00680F781E02DB0
:1021E000099408952091700130917101821793072D
:1021F00071F09093710180937001E0917401F091FE
:102200007501309721F00084F185E02D099408953F
:1022100008950C9408110E94621C0E94AD030C9456
:10222000241D9F92AF92BF92CF92DF92EF92FF92C6
:102230000F931F93CF93DF9300D000D000D0CDB782
:10224000DEB70E94C5030DE010E0AA24A394B12CD0
:10225000902E802F0E94B304980129583E4F6901A7
:10226000F901F080F826A1F40150110988F78FEFE9
:1022700089838A831B820E946B1C8160782F9D83D7
:102280008C8349815A816B818D810E94A8112FC056
:102290009091DA0191FF04C08E830E94B9048E816F
:1022A00025E030E0A501022E01C0440F0A94EAF7B0
:1022B000E42E4F21C1F029839A828E2191E009F406
:1022C00090E09B830E946B1C8160782F9D838C83A0
:1022D00049815A816B818D810E94A811F60180810C
:1022E000E826E08204C021503109E0F6BDCF0E940B
:1022F0000B20109176010E94BA101817B9F00E94B5
:10230000BA108093760126960FB6F894DEBF0FBE02
:10231000CDBFDF91CF911F910F91FF90EF90DF9094
:10232000CF90BF90AF909F900C94B30926960FB6B4
:10233000F894DEBF0FBECDBFDF91CF911F910F91FB
:10234000FF90EF90DF90CF90BF90AF909F90089557
:10235000CF93DF93CDB7DEB72B970FB6F894DEBFE0
:102360000FBECDBF4F83588769877A878B87DE0181
:10237000119686E0FD0111928A95E9F785E0FE014C
:10238000379601900D928A95E1F749815A816B81C8
:102390007C818D819E810E94F1172B960FB6F89457
:1023A000DEBF0FBECDBFDF91CF910895CF938823BD
:1023B00009F4C2C0C82F823859F40E94BA1081FDB6
:1023C000BBC089E30E94CB1A0E94981B89E30CC012
:1023D000833879F40E94BA1080FDAEC083E50E9474
:1023E000CB1A0E94981B83E50E940D1BCF910C9481
:1023F000981B843859F40E94BA1082FD9DC087E46E
:102400000E94CB1A0E94981B87E4EECF8CEF8C0FB2
:10241000813A48F48C2F0E944E2281118DC08C2F5E
:102420000E94CB1AE3CF80E28C0F883048F4C7704B
:1024300081E001C0880FCA95EAF70E94511BD6CFF0
:102440008BE58C0F833078F4C53A29F0C63A31F029
:1024500083E890E005C081E890E002C082E890E067
:10246000CF910C94DC1088E58C0F833108F064C0A8
:10247000C83A39F1C93A41F1CA3A49F1CB3A51F176
:10248000CC3A59F1CD3A61F1C03B69F1CE3A71F1E4
:10249000CF3A79F1C13B81F1C23B89F1C33B91F164
:1024A000C43B99F1C53BA1F1C63BA9F1C73BB1F1D2
:1024B000C83BB9F1C93BC1F1CA3BC9F180E090E02A
:1024C00038C082EE90E035C089EE90E032C08AEEEE
:1024D00090E02FC085EB90E02CC086EB90E029C007
:1024E00087EB90E026C08CEC90E023C08DEC90E070
:1024F00020C083E891E01DC08AE891E01AC082E91B
:1025000091E017C084E991E014C081E292E011C02B
:1025100083E292E00EC084E292E00BC085E292E09A
:1025200008C086E292E005C087E292E002C08AE23B
:1025300092E0CF910C94F210CF910895882309F482
:102540004BC0823859F40E94BA1081FF45C089E31C
:102550000E94CB1A0E94981B89E30CC0833871F447
:102560000E94BA1080FF38C083E50E94CB1A0E94F7
:10257000981B83E50E940D1B0C94981B843859F41A
:102580000E94BA1082FF28C087E40E94CB1A0E94E2
:10259000981B87E4EFCF9CEF980F913A58F390E2A5
:1025A000980F983050F4877091E001C0990F8A9588
:1025B000EAF7892F0E94571BDFCF9BE5980F9330D6
:1025C00020F480E090E00C94DC10885A833120F4F1
:1025D00080E090E00C94F2100895882321F00E948E
:1025E000511B0C94981B0895882321F00E94571BBF
:1025F0000C94981B08957F928F929F92AF92BF92F6
:10260000CF92DF92EF92FF920F931F93CF93DF93BE
:102610001F92CDB7DEB77C01C62E772EFC01058157
:1026200002950F70128111110E946E1B0E94C41A34
:10263000882379F0112369F080E28C0D883048F00E
:1026400082E00E94AD1A0E94C41A91E0D82ED926C9
:1026500001C0D12CE72DE295EF70F0E0E059FF4F7B
:102660000C948324872D807F072D0F70882311F011
:102670000295007F112389F0002309F490C180E2C4
:102680008C0D883020F4802F0E94511B03C0802FB6
:102690000E94611B0E94981B82C18C2D0E949E1279
:1026A000002309F495C180E28C0D883020F4802F3E
:1026B0000E94571B03C0802F0E94671B0E94981B1B
:1026C00087C1972D907F872D8F70903211F0829562
:1026D000807FCC2021F0F1E0CF16B1F01EC0112395
:1026E00049F0002309F414C1013009F011C10E941E
:1026F000811B6EC1002319F0013009F469C189837F
:102700000E94841B89810AC1112321F0023008F044
:102710005FC1FEC001115CC101C1112321F0002382
:1027200009F4F6C03CC1002309F4F8C03EC1872D6E
:1027300086958695837090E0009719F0019761F077
:1027400047C1112321F08C2D972D937002C080E09A
:1027500090E00E94DC103CC1112321F08C2D972DBC
:10276000937002C080E090E00E94F21031C18C2D85
:10277000112319F00E94131F02C00E947B1F0E94A8
:10278000002026C1872D837009F052C0111120C18D
:102790008C2D829586958770880F880F9C2D9F7051
:1027A000892E912CA12CB12C082E04C0880C991CC8
:1027B000AA1CBB1C0A94D2F7C4FE14C00FE010E0A0
:1027C00020E030E0B901A80104C0440F551F661F86
:1027D000771F8A95D2F7CB01BA01609570958095E5
:1027E000909503C060E070E0CB01272D26952695DB
:1027F000237030E02230310569F02330310589F053
:10280000682979298A299B292130310571F00E9494
:102810003919DEC0682979298A299B290E9455190E
:10282000D7C00E943919C501B4010E941D19D0C03A
:10283000112319F0872D817001C08695882309F432
:10284000C7C08C2D829586958770880F880F9C2D28
:102850009F70892E912CA12CB12C082E04C0880CBD
:10286000991CAA1CBB1C0A94D2F7C4FE14C00FE02A
:1028700010E020E030E0B901A80104C0440F551F6A
:10288000661F771F8A95D2F7CB01BA0160957095C4
:102890008095909503C060E070E0CB01272D2695D0
:1028A00026952370422F50E04230510569F04330A5
:1028B000510589F0682979298A299B2941305105D8
:1028C00071F00E94131A84C0682979298A299B29EA
:1028D0000E942F1A7DC00E94131AC501B4010E94E4
:1028E000F71976C08C2D90E0FC01E05EF109E5312E
:1028F000F10508F050C0E058FF4F0C9483240C2DD4
:102900000F70872D8F71112331F00E949019802F45
:102910000E94ED125DC00E94B119802F0E94F41236
:1029200057C0112339F0011153C0872D8F710E94B8
:10293000D6194EC0023008F04BC0F7CF112339F042
:10294000872D8F710E94901943C01123C9F3872DE1
:102950008F710E94B1193CC0112329F0872D8F710E
:102960000E947B1935C00E94711932C0112351F0A9
:10297000172D1F71812F0E94901963E0812F0E94F3
:10298000A41A26C081E00E94AD1A023008F182E04C
:102990000E94AD1A1DC0112331F0002389F28C2D45
:1029A0000E94D61115C0002391F28C2D0E949E1218
:1029B0000FC0472D4F706C2DC7010E948F050E94DC
:1029C000951806C0472D4F706C2DC7010E94C20696
:1029D000DD20F9F00E94A01A80FD1BC0F7011282D1
:1029E0000E949A1A0E949019C7010E9418150E940D
:1029F0009A1A0F90DF91CF911F910F91FF90EF9056
:102A0000DF90CF90BF90AF909F908F907F900C946D
:102A1000B1190F90DF91CF911F910F91FF90EF901F
:102A2000DF90CF90BF90AF909F908F907F90089550
:102A30000F931F93CF93DF93EC01888199812B81B2
:102A40003C81232BB9F09F3F11F48F3F99F0CE01C9
:102A50000E941A06882371F0688179818A810E9418
:102A6000961A8C010E944B1A0E941219B801CE01CD
:102A70000E94FB12DF91CF911F910F9108950E9448
:102A80006E1B0E947E1B0E94431B0E94981B0E948B
:102A9000B1200E94002080E090E00E94DC1080E0E5
:102AA00090E00C94F2100E945E1B0C943F150E9463
:102AB0008B1A292F22952F7030E02C3031054CF4E1
:102AC0002A3031056CF42250310922303105A8F446
:102AD00007C02C30310569F02F30310551F00DC0A1
:102AE000803F69F018F4803E40F409C0843F29F427
:102AF00006C093FB882780F9089580E0089581E05F
:102B00000895CF93DF9300D000D01F92CDB7DEB7EA
:102B10000F900F900F900F900F90DF91CF9108952D
:102B2000CF93DF9300D000D000D0CDB7DEB726968C
:102B30000FB6F894DEBF0FBECDBFDF91CF910895E1
:102B40001F93CF93DF93C091850116E0809186019A
:102B5000C81799F0D0E01C9FF0011D9FF00D1124C3
:102B6000E957FE4F40815181628173818481958153
:102B70000E9490152196C770E9CFDF91CF911F91E8
:102B800008954091B7015091B8016091B9017091D9
:102B9000BA018091BB019091BC010C949015809179
:102BA000BC0182958F7009F054C08091B9018823CF
:102BB00009F44FC080918501A09186016091B70111
:102BC0007091B8014091BA015091BB01B6E08A17EB
:102BD00009F43FC090E041155105C1F17F3F11F468
:102BE0006F3FA1F1B89FF001B99FF00D1124E95793
:102BF000FE4F218172132AC02081621327C02281D7
:102C0000211124C0238134812417350710F4215069
:102C10003109241B350B283C3105C0F42091BC013F
:102C20002F7020612093BC0126E0289FF001299F8E
:102C3000F00D1124E457FE4F80818F7080618083F6
:102C400087EB91E00E9418150C94A01501968770EF
:102C5000BECF0895CF92DF92EF92FF920F931F9312
:102C6000CF93DF93CDB7DEB762970FB6F894DEBF90
:102C70000FBECDBF8C0185E0F801DE011D960190ED
:102C80000D928A95E1F7D8014C9111965C911197BC
:102C900012966C9112971396CD90DC901497309108
:102CA000B7017091B8018091BA019091BB01009772
:102CB00009F46BC17F3F19F43F3F09F466C1E0900E
:102CC000B901EE2009F4C0C02091BC01C816D90694
:102CD00028F0F601E81BF90BCF0104C08095909510
:102CE0008C0D9D1DFF24F394883C910578F0F12C08
:102CF000207F09F0C6C07C2DD98AC88A89890E94A4
:102D0000811587EB91E00E941815B1C0822F807F5A
:102D100009F046C0751314C0341312C0611110C0FD
:102D20002F7020612093BC010E94C11587EB91E0B8
:102D30000E9418158091BC01D80115968C932EC065
:102D4000CD2819F15F3F11F44F3FF9F0F62E6111D4
:102D50001CC0809185012091860136E0821709F41C
:102D60005AC090E0389FF001399FF00D1124E957C7
:102D7000FE4F7181571306C07081471303C07281E3
:102D8000711103C001968770E9CFF62E662309F40E
:102D900018C18091BC0181608093BC01F12C11C1EC
:102DA000751308C0341306C0611104C08091BC01C2
:102DB000D801C3C04D875E878D859E856A8B0E9432
:102DC00057156A898823E1F16623D1F12091BC016E
:102DD000822F82958F7090E0029774F08091B701F6
:102DE0009091B80198878F831986DB86CA862C87D5
:102DF000CE0107960E94181586E0F801A7EBB1E016
:102E000001900D928A95E1F70E94CF150E94C1159D
:102E1000FF24F394D6C04D875E878D859E850E94E2
:102E20008B1A292F22952F7030E0223031050CF0BB
:102E3000BCC09F7009F0B6C0805E883008F4C1C085
:102E4000C8010E941815E4CFC816D90608F453C06B
:102E5000F601E81BF90BCF01883C910508F450C03E
:102E6000F12C7C2DD98AC88A89890E948115E7EBCB
:102E7000F1E086E0DF011D928A95E9F70E94C11515
:102E8000A0C0751314C0341312C0611110C080911A
:102E9000BC01F8018583C8010E94181586E0E7EBA4
:102EA000F1E0DF011D928A95E9F7FE2C8AC04D877B
:102EB0005E878D859E856A8B0E9457156A89882357
:102EC00009F4BECF662309F4BBCF2091BC01822F49
:102ED00082958F7090E002970CF48ECF8091B701AD
:102EE0009091B8019A8389831B82DD82CC822E83E4
:102EF000CE0101967FCF809590958C0D9D1DACCF16
:102F0000F62E662309F49CCF75132EC034132CC003
:102F10002091BC0120FD1FC0822F82958F70D9F0B7
:102F2000D80115962C9315978F3049F08F5F982F05
:102F30009295907F822F8F70892B15968C93C80164
:102F40000E94181586E0F801A7EBB1E001900D9200
:102F50008A95E1F793CF86E0F801A7EBB1E0019005
:102F60000D928A95E1F72DC04D875E878D859E85F0
:102F70000E945715811140CF8091BC0181608093E0
:102F8000BC01C8010E9418151CC0662309F458CF63
:102F90004D875E878D859E850E945715882309F48D
:102FA0004FCF2ACF811148CF0CC0243031050CF00F
:102FB00047CF9F7009F440CFF8019581907F09F0C9
:102FC0003BCF8F2D62960FB6F894DEBF0FBECDBFFC
:102FD000DF91CF911F910F91FF90EF90DF90CF90F5
:102FE00008951F93CF93DF93CDB7DEB72C970FB61D
:102FF000F894DEBF0FBECDBF4F83588769877A87AD
:103000008B879C87CE0107960E942A16882369F039
:103010008F8198852A853B85232BF1F19F3F09F00D
:1030200063C08F3F09F060C037C086E0FE0137966D
:10303000DE01119601900D928A95E1F76F817885F6
:10304000EA85FB85309741F17F3F11F46F3F21F115
:103050002091860130E0C90101968770992740913F
:10306000850150E08417950709F447C069837A8386
:10307000FD83EC8396E0929FD001939FB00D1124C5
:10308000A957BE4FFE01319601900D929A95E1F736
:10309000809386010E94A01516E080918501909191
:1030A00086018917C1F1189FC001112489579E4FCD
:1030B0000E942A16882379F1E09185011E9FF00174
:1030C0001124E957FE4F40815181628173818481CF
:1030D00095810E9490158091850190E001968770FE
:1030E000992780938501D9CF4F81588569857A8545
:1030F0008B859C850E949015CFCF0E94531510920E
:10310000860110928501E7EBF1E086E0DF011D9278
:103110008A95E9F7C1CF2C960FB6F894DEBF0FBEA3
:10312000CDBFDF91CF911F910895EF92FF920F9342
:103130001F93CF93DF938C01009709F46CC0F12C9F
:10314000EE24E394E8012196F8018491843740F459
:10315000843008F051C0813081F0823019F15BC0B9
:10316000853709F444C0A8F19CE7980F903708F020
:1031700052C08F770E949E1241C00E5F1F4FFE010A
:10318000C49180E28C0F883048F4C7708E2D01C046
:10319000880FCA95EAF70E94711B14C08C2F0E94F9
:1031A000D6112DC00E5F1F4FFE01C49180E28C0F1F
:1031B000883058F4C7708E2D01C0880FCA95EAF781
:1031C0000E94771B0E94981B1AC08C2F0E949E128F
:1031D00016C00E5F1F4FFE01C491CC2381F08FE912
:1031E0009FE00197F1F700C00000C150F6CF0E5FDD
:1031F0001F4FFE01F49003C00E94D6118E018F2D47
:10320000882309F49FCFEFE9FFE03197F1F700C081
:1032100000008150F5CFDF91CF911F910F91FF906A
:10322000EF90089508956093C1017093C201809357
:10323000C3019093C4010C943F150F931F93009109
:10324000C1011091C2012091C3013091C401DC0180
:10325000CB01802B912BA22BB32B8093C101909398
:10326000C201A093C301B093C4011F910F910C94AC
:103270003F150F931F930091C1011091C20120913E
:10328000C3013091C401DC01CB0180239123A2232F
:10329000B3238093C1019093C201A093C301B09363
:1032A000C4011F910F910C943F150F931F93009130
:1032B000C1011091C2012091C3013091C401DC0110
:1032C000CB0180279127A227B3278093C101909338
:1032D000C201A093C301B093C4011F910F910C943C
:1032E0003F151092BD011092BE011092BF011092C5
:1032F000C0010C943F1541E050E060E070E004C074
:10330000440F551F661F771F8A95D2F74093BD0162
:103310005093BE016093BF017093C0010C943F15A0
:1033200041E050E060E070E004C0440F551F661FAC
:10333000771F8A95D2F78091BD019091BE01A0912F
:10334000BF01B091C001482B592B6A2B7B2B4093B6
:10335000BD015093BE016093BF017093C0010C94F6
:103360003F1541E050E060E070E004C0440F551F9D
:10337000661F771F8A95D2F7409550956095709596
:103380008091BD019091BE01A091BF01B091C0019B
:10339000482359236A237B234093BD015093BE01E8
:1033A0006093BF017093C0010C943F1541E050E061
:1033B00060E070E004C0440F551F661F771F8A95B8
:1033C000D2F78091BD019091BE01A091BF01B09153
:1033D000C001482759276A277B274093BD01509396
:1033E000BE016093BF017093C0010C943F150F9311
:1033F0001F930091BD011091BE012091BF0130913A
:10340000C001DC01CB01802B912BA22BB32B80932D
:10341000BD019093BE01A093BF01B093C0011F9165
:103420000F910C943F150F931F930091BD011091C4
:10343000BE012091BF013091C001DC01CB0180238E
:103440009123A223B3238093BD019093BE01A09347
:10345000BF01B093C0011F910F910C943F150F93C2
:103460001F930091BD011091BE012091BF013091C9
:10347000C001DC01CB0180279127A227B3278093CD
:10348000BD019093BE01A093BF01B093C0011F91F5
:103490000F910C943F150895CF92DF92EF92FF9217
:1034A0000F931F93CF93DF938C01C090C101D090F5
:1034B000C201E090C301F090C4018091BD019091E0
:1034C000BE01A091BF01B091C001C82AD92AEA2A41
:1034D000FB2ACFE1D0E0D701C6010C2E04C0B6957F
:1034E000A795979587950A94D2F780FF06C0B801F3
:1034F0008C2F0E941809019721F4219760F780E032
:1035000001C08C2FDF91CF911F910F91FF90EF9011
:10351000DF90CF900895CF93DF93EC010E944C1A77
:10352000BE010E941809DF91CF910895CB010E943E
:103530008B1A08958091C501859585958595089587
:103540008091C5018770089598E0899F90011124AA
:10355000262B2093C5010C9490192091C5018095CC
:1035600082238093C501982F977069F430E0482F2B
:10357000552747FD50952417350729F085958595E2
:1035800085950C94B11908959091C501977081E0CB
:1035900009F480E0089590910C01992321F0909115
:1035A0000D01911109C020910E0130910F01F90117
:1035B00032969FEF40E01FC0982F9695969596956E
:1035C0009F3050F5E0910E01F0910F01E90FF11DD0
:1035D000877021E030E0A90102C0440F551F8A9591
:1035E000E2F7CA019181892B818308959F3F39F0C9
:1035F0004F5F4E3041F051915813F8CF0DC051112B
:10360000F7CF942FF5CF9F3F39F0F901E90FF11D66
:1036100097FDFA9582830895089590910C0199235E
:1036200021F090910D01911109C020910E0130916E
:103630000F01F9013296205F3F4F1FC0982F9695DA
:10364000969596959F30F0F4E0910E01F0910F0160
:10365000E90FF11D877021E030E0A90102C0440F9D
:10366000551F8A95E2F7CA0180959181892381834C
:1036700008953196E217F30729F090819813F9CF56
:103680001082F7CF089581E090E0E0910E01F09173
:103690000F01E80FF91F1082019680319105A9F7FB
:1036A00008959091D901892B8093D901089580952F
:1036B0009091D90189238093D90108951092D9015D
:1036C00008959091D801892B8093D8010895809511
:1036D0009091D80189238093D80108951092D80140
:1036E00008959091D701892B8093D70108958095F3
:1036F0009091D70189238093D70108951092D70123
:1037000008958093C60108951092C601089580918E
:103710000E0190910F01FC0131969C01205F3F4FFB
:1037200080E0919191118F5FE217F307D1F708952F
:10373000E0910E01F0910F018091D9018083E09119
:103740000E01F0910F0190818091D801892B808327
:10375000E0910E01F0910F0190818091D701892BAA
:1037600080838091C601882361F0E0910E01F09181
:103770000F019081892B80830E94871B81111092F9
:10378000C60180910E0190910F010C94C61020E0AB
:10379000009739F0AC0141505109842395232F5FE4
:1037A000F7CF822F0895CF92DF92EF92FF926C01B4
:1037B000EE24FF24C114D104E104F10421F0C70177
:1037C000B60120E101C020E0C72ED82EE92EFF244B
:1037D000C114D104E104F10419F0285FC701B60156
:1037E0006B017C0154E0F694E794D794C7945A9502
:1037F000D1F7C114D104E104F10419F02C5FC70121
:10380000B6016B017C0142E0F694E794D794C7942B
:103810004A95D1F7C114D104E104F10419F02E5FE7
:10382000C701B601DC01CB01B695A79597958795A1
:10383000892B8A2B8B2B09F02F5F822FFF90EF9023
:10384000DF90CF9008958091F101843021F11092A2
:10385000DB0120E488E190E00FB6F894A89580930E
:1038600060000FBE2093600080E00E94B30983B720
:10387000817F846083BF83B7816083BF789488959C
:1038800083B78E7F83BF88E10FB6F8948093600082
:10389000109260000FBE0895089508950E944C1C78
:1038A0000E94C5030E944D1C0E94BA0491E0811140
:1038B00001C090E0892F08950E9453150E94BA100C
:1038C0000C94B30982E084BD93E095BD9AEF97BD57
:1038D00080936E0008952FB7F8948091DC01909149
:1038E000DD01A091DE01B091DF012FBF0895CF92DD
:1038F000DF92EF92FF920F931F932FB7F8944091AE
:10390000DC015091DD016091DE017091DF012FBF7C
:103910006A017B01EE24FF248C0120E030E0C01618
:10392000D106E206F30610F4415051099A01281B12
:10393000390BC9011F910F91FF90EF90DF90CF904D
:1039400008951F920F920FB60F9211248F939F9399
:10395000AF93BF938091DC019091DD01A091DE01D6
:10396000B091DF010196A11DB11D8093DC01909300
:10397000DD01A093DE01B093DF01BF91AF919F9174
:103980008F910F900FBE0F901F9018950E94B70D4A
:10399000F8942FEF87EA91E6215080409040E1F7BC
:1039A00000C0000087E090EBDC018093FB01909366
:1039B000FC01A093FD01B093FE019CE088E10FB6ED
:1039C000F894A895809360000FBE90936000FFCF9D
:1039D000EF92FF920F931F93CF93DF93D82FCDE0F9
:1039E0008C2F0E94B30405E010E0E82EF12CC701F3
:1039F000002E02C0959587950A94E2F780FF09C0D2
:103A0000602F7C2F80E00E94C306D81302C081E0A3
:103A100006C00150110958F7C15010F780E0DF913E
:103A2000CF911F910F91FF90EF900895CF93C82FE2
:103A30008CE20E94E81C882321F08C2FCF910C94FB
:103A4000E81C80E0CF910895CF930E946B1E8111F6
:103A500002C00E94511EC5E6C15049F00E94C50334
:103A60008FE39CE90197F1F700C00000F5CF89E2F0
:103A70000E94161D811113C18AE20E94161D811138
:103A80000E94511E85E00E94161D81110E94C61CD5
:103A90000E94761E8093DA0187E00E94161D88231B
:103AA000A9F18BE10E94161D882351F08091DA0163
:103AB00081FB222720F991E0922790FB81F90EC02B
:103AC0008EE00E94161D882361F08091DA0182FB4E
:103AD000222720F991E0922790FB82F98093DA0166
:103AE00015C080E10E94161D9091DA01882341F0F3
:103AF00093FB222720F981E0822780FB93F904C001
:103B0000892F809580FB90F99093DA018091DA01FA
:103B10000E947A1E0E94881E8093FA0180EE0E9405
:103B2000161D882341F08091FA01982F909590FB03
:103B300080F98093FA0189E30E94161D882359F0C9
:103B40008091FA0181FB222720F991E0922790FBD6
:103B500081F98093FA0182EE0E94161D882359F0A4
:103B60008091FA0182FB222720F991E0922790FBB5
:103B700082F98093FA0186EE0E94161D882359F07F
:103B80008091FA0183FB222720F991E0922790FB94
:103B900083F98093FA0183EE0E94161D882359F061
:103BA0008091FA0184FB222720F991E0922790FB73
:103BB00084F98093FA0185E30E94161D882359F049
:103BC0008091FA0185FB222720F991E0922790FB52
:103BD00085F98093FA0181E30E94161D882359F02C
:103BE0008091FA0186FB222720F991E0922790FB31
:103BF00086F98093FA0181E10E94161D882359F00D
:103C00008091FA0187FB222720F991E0922790FB0F
:103C100087F98093FA018091FA010E948C1E8091AD
:103C2000FA0187FB882780F980930D0187E20E94C3
:103C3000161DC82F8EE10E94161D8111C2608FE1F2
:103C40000E94161D8111C46080E20E94161D811120
:103C5000C86081E20E94161D8111C06182E20E944B
:103C6000161D8111C06283E20E94161D8111C0647D
:103C700084E20E94161D882311F0C06802C0CC2384
:103C800029F08C2F0E94831E6C2F03C00E947F1E80
:103C9000682F70E080E090E0CF910C941319CF91E1
:103CA00008956DEE7EEF80E090E00E94BD2460E01C
:103CB00082E090E00E94AB2460E083E090E00E940C
:103CC000AB2460E084E090E00E94AB2460E085E0FB
:103CD00090E00C94AB2480E090E00E94A52421E0C9
:103CE0008D3E9E4F09F020E0822F089582E090E003
:103CF0000C949D24682F82E090E00C94AB2483E028
:103D000090E00C949D24682F83E090E00C94AB2409
:103D100084E090E00C949D24682F84E090E00C9463
:103D2000AB248091E20180FF0BC06091130185E01C
:103D3000689FB001112475956795759567952BC09F
:103D400081FF09C06091130185E0689FB0011124D3
:103D50007595679520C082FF07C06091130185E0CB
:103D6000689FB001112417C09091E3019923D1F00D
:103D700060911201961788F72091130185E0289F22
:103D800090011124929FA001939F500D112470E087
:103D9000CA010E946F246038710540F461157105F5
:103DA00039F002C065E070E0862F08958FE708952E
:103DB00081E008958091E20180FF08C060911101C7
:103DC00070E0759567957595679521C081FF06C070
:103DD0006091110170E07595679519C082FF04C06C
:103DE0006091110170E010C09091E3019923C1F03E
:103DF000609110019617A0F780911101899FC00171
:103E0000112470E00E946F246038710528F4611558
:103E1000710521F0862F08958FE7089581E00895B8
:103E200061E070E0F4CF803F21F40E94911E819503
:103E300004C0813F29F40E94911E8093E6010895F9
:103E4000823F21F40E94911E819504C0833F29F492
:103E50000E94911E8093E5010895893F19F40E9404
:103E6000DA1E05C08A3F31F40E94DA1E81958093E4
:103E7000E70108958B3F21F40E94DA1E819504C06A
:103E80008C3F29F40E94DA1E8093E8010895843F54
:103E900021F48091E401816017C0853F21F4809175
:103EA000E401826011C0863F21F48091E4018460C6
:103EB0000BC0873F21F48091E401886005C0883FF2
:103EC00031F48091E40180618093E40108958D3F95
:103ED00021F48091E20181600BC08E3F21F480913A
:103EE000E201826005C08F3F29F48091E201846085
:103EF0008093E2010895803F39F48091E60187FFC5
:103F00006CC01092E60169C0813F29F48091E601FE
:103F10001816BCF362C09091E501823F29F497FF27
:103F20005CC01092E50159C0833F19F41916CCF317
:103F300054C0893F41F48091E70118160CF04DC040
:103F40001092E7014AC08A3F29F48091E70187FF78
:103F500044C0F6CF8B3F39F48091E80187FF3DC024
:103F60001092E8013AC08C3F29F48091E8011816BC
:103F7000BCF333C0843F21F48091E4018E7F17C0ED
:103F8000853F21F48091E4018D7F11C0863F21F4AB
:103F90008091E4018B7F0BC0873F21F48091E40185
:103FA000877F05C0883F31F48091E4018F7E809344
:103FB000E40113C08D3F21F48091E2018E7F0BC09C
:103FC0008E3F21F48091E2018D7F05C08F3F29F45F
:103FD0008091E2018B7F8093E2018091E501811164
:103FE0000EC08091E60181110AC08091E701811124
:103FF00006C08091E801811102C01092E30108958A
:1040000084EE91E00E94D1100E946B1C9093E1011C
:104010008093E00108951F93CF93DF938091E00197
:104020009091E1010E94771CAC019091E3019923EA
:1040300021F02091140130E006C0209115018AE0A2
:10404000289F900111244217530708F486C08091DD
:10405000E501C091E601D091E7011091E8018111DD
:1040600007C0C11176C0D11174C0111172C075C0E2
:104070009F3F19F09F5F9093E301181624F40E946C
:10408000911E8093E5018091E50187FF05C00E94A4
:10409000911E81958093E5011C1624F40E94911EC7
:1040A0008093E6018091E60187FF05C00E94911E82
:1040B00081958093E6016091E501662339F1C09115
:1040C000E601CC2319F1772767FD7095872F972F8D
:1040D0000E94802323E333E343E35FE30E94E4236E
:1040E0000E944D236093E5016C2F772767FD709543
:1040F000872F972F0E94802323E333E343E35FE37B
:104100000E94E4230E944D236093E6011D1624F4CF
:104110000E94DA1E8093E7018091E70187FF05C0C6
:104120000E94DA1E81958093E701111624F40E9403
:10413000DA1E8093E8018091E80187FF05C00E94A4
:10414000DA1E81958093E801DF91CF911F910C9445
:1041500000209F3F09F08ECF96CFDF91CF911F9126
:104160000895E4EEF1E085E0DF011D928A95E9F71C
:104170001092E3011092E2010895833081F128F456
:10418000813059F08230D1F00895853009F449C06A
:10419000B8F1863009F456C0089580911501262F94
:1041A00030E0280F311D2F3F310524F4680F609354
:1041B000150108958FEF80931501089580911401E2
:1041C000262F30E0280F311D2F3F310524F4680FD2
:1041D0006093140108958FEF8093140108958091E6
:1041E0001301262F30E0280F311D2F3F310524F415
:1041F000680F6093130108958FEF80931301089562
:1042000080911201262F30E0280F311D2F3F3105FC
:1042100024F4680F6093120108958FEF80931201C8
:10422000089580911101262F30E0280F311D2F3F76
:10423000310524F4680F6093110108958FEF809386
:104240001101089580911001262F30E0280F311DB3
:104250002F3F310524F4680F6093100108958FEF0C
:10426000809310010895833011F128F4813049F0D2
:10427000823091F00895853081F120F18630C1F1CE
:10428000089580911501681720F4861B809315010D
:10429000089510921501089580911401681720F473
:1042A000861B809314010895109214010895809143
:1042B0001301681720F4861B809313010895109250
:1042C0001301089580911201681720F4861B8093D2
:1042D000120108951092120108958091110168173A
:1042E00020F4861B80931101089510921101089506
:1042F00080911001681720F4861B809310010895A7
:104300001092100108950F931F938D3109F46BC023
:1043100008F03FC08E3009F47FC0C0F4873009F444
:1043200069C068F4863009F0B1C08091DA01817FFC
:104330008E7F8093DA0181E08093EA01A8C0883003
:1043400009F4A2C08B3009F49FC0A0C0863109F4E3
:104350009BC078F4803109F472C0813109F096C0B5
:104360000E94531590910D0181E0892780930D01E2
:104370008BC0893109F488C08B3109F087C08091E6
:10438000DA0181FB222720F991E0922790FB81F945
:104390004CC0853309F470C048F4873209F46CC00E
:1043A00008F459C0893209F467C070C0833438F406
:1043B0008A3308F04EC0883309F466C067C083347E
:1043C00009F45AC0883409F061C00E9453150FEFF8
:1043D00013ED20E3015010402040E1F700C0000041
:1043E0000E94C61C51C00E9407230E94BA100E945E
:1043F000B3094AC09091DA01892F8095817080FBC2
:1044000090F929F0966098609093DA0140C0997F06
:10441000977F9093DA0138C08091DA0182FB2227DE
:1044200020F991E0922790FB82F98093DA01992399
:1044300059F18091DA0181608093DA0125C0809181
:10444000DA0183FB222720F991E0922790FB83F980
:10445000ECCF895301C08D5141E050E060E070E045
:104460008A019B0104C0000F111F221F331F8A9570
:10447000D2F7C901B80104C061E070E080E090E0CB
:104480000E9413190E94531581E001C080E01F9122
:104490000F91089580E0089580E00895CF93C82F8C
:1044A0008091EA01813079F018F08230E9F187C01B
:1044B000E0910E01F0910F018081813169F082322B
:1044C00009F07FC009C0E0910E01F0910F018081D9
:1044D000813111F0823261F48C2F0E944A228111C5
:1044E00004C08C2F0E9483211DC081E090E01AC07F
:1044F0008C2F0E944C22811114C0C43179F048F4F1
:10450000CB3079F0C03109F060C082E08093EA01DD
:1045100008C0C93219F0C83321F057C01092EA011F
:1045200054C081E0817053C0C93289F118F5C4319B
:1045300071F1A8F4C73009F046C08AE080931501F4
:1045400094E19093140193E09093130180931201EE
:1045500088E08093110188E28093100134C0CE512D
:10456000C63088F5EC2FF0E0E65DFE4F8081809349
:10457000E90129C0CE34E9F020F4CB3421F56AE01A
:1045800013C0C13579F0C235F1F461E00DC08091FE
:10459000E901882319F01092E90115C081E08093A8
:1045A000EA0115C061E006C08091E9010E94BD20CA
:1045B0000AC06AE08091E9010E94332104C0109290
:1045C000EA0180E004C081E002C080E0ABCFCF917F
:1045D0000895E1E8F0E080818860808380818160D7
:1045E00080838FB7F89493E09093890090ED909337
:1045F00088008FBF0895EFE6F0E0808182608083BD
:104600000895EFE6F0E080818D7F80830895EFE6E6
:10461000F0E0908182E08927808308951F920F92B5
:104620000FB60F9211242F933F934F935F936F9385
:104630007F938F939F93AF93BF93EF93FF9380915B
:10464000EB019091EC0101969093EC018093EB01CA
:10465000811103C082E00E94B309E091EC01E6956C
:10466000E695F0E0E855FA4FE4918091EB018E1366
:1046700003C080E00E94B309FF91EF91BF91AF9119
:104680009F918F917F916F915F914F913F912F916A
:104690000F900FBE0F901F90189504D06894B11121
:1046A0008DC0089570D088F09F5790F0B92F99274A
:1046B000B751A0F0D1F0660F771F881F991F1AF02D
:1046C000BA95C9F712C0B13081F077D0B1E0089542
:1046D00074C0672F782F8827B85F39F0B93FCCF3C3
:1046E000869577956795B395D9F73EF49095809523
:1046F000709561957F4F8F4F9F4F0895E89409C043
:1047000097FB3EF490958095709561957F4F8F4F04
:104710009F4F9923A9F0F92F96E9BB279395F6951A
:10472000879577956795B795F111F8CFFAF4BB0F98
:1047300011F460FF1BC06F5F7F4F8F4F9F4F16C0FC
:10474000882311F096E911C0772321F09EE8872F86
:10475000762F05C0662371F096E8862F70E060E042
:104760002AF09A95660F771F881FDAF7880F9695BB
:10477000879597F9089557FD9058440F551F59F0A4
:104780005F3F71F04795880F97FB991F61F09F3F3E
:1047900079F087950895121613061406551FF2CF67
:1047A0004695F1DF08C0161617061806991FF1CFB7
:1047B00086957105610508940895E894BB276627DE
:1047C0007727CB0197F908950BD078C069D028F0EE
:1047D0006ED018F0952309F05AC05FC01124EECFB7
:1047E000CADFA0F3959FD1F3950F50E0551F629F4C
:1047F000F001729FBB27F00DB11D639FAA27F00D3A
:10480000B11DAA1F649F6627B00DA11D661F829F60
:104810002227B00DA11D621F739FB00DA11D621F45
:10482000839FA00D611D221F749F3327A00D611D62
:10483000231F849F600D211D822F762F6A2F112444
:104840009F5750408AF0E1F088234AF0EE0FFF1F97
:10485000BB1F661F771F881F91505040A9F79E3FCE
:10486000510570F014C0AACF5F3FECF3983EDCF323
:10487000869577956795B795F795E7959F5FC1F70B
:10488000FE2B880F911D9695879597F9089597F9B6
:104890009F6780E870E060E008959FEF80EC0895E6
:1048A00000240A941616170618060906089500240F
:1048B0000A9412161306140605060895092E039489
:1048C000000C11F4882352F0BB0F40F4BF2B11F4FD
:1048D00060FF04C06F5F7F4F8F4F9F4F089597FB1E
:1048E000072E16F4009407D077FD09D00E94892482
:1048F00007FC05D03EF4909581959F4F08957095E3
:1049000061957F4F0895EE0FFF1F0590F491E02D04
:104910000994AA1BBB1B51E107C0AA1FBB1FA61706
:10492000B70710F0A61BB70B881F991F5A95A9F758
:1049300080959095BC01CD010895F999FECF92BD67
:1049400081BDF89A992780B50895A8E1B0E042E0CA
:1049500050E00C94C524262FF999FECF92BD81BD5D
:10496000F89A019700B4021639F01FBA20BD0FB6AD
:10497000F894FA9AF99A0FBE08950196272F0E948B
:10498000AC240C94AB24DC01CB01FC01F999FECFE3
:1049900006C0F2BDE1BDF89A319600B40D924150C7
:0A49A0005040B8F70895F894FFCFD7
:1049AA000220B509430A200AEC09B8090101C70126
:1049BA0028080A03140A3F4D363969051C05E6041E
:1049CA00AD044004590472048B0401020304050671
:0449DA0007080900C1
:00000001FF
